:020000040000FA
:0400000072303A28F8
:040004000034003490
:08000800A000030EA100831209
:1000100081018B100B11210E8300A00E200E090010
:0C007400203084008001840A80300402E7
:10008000031C3C28302183160C3085058701831220
:10009000850187010730990000309A0010308316DF
:1000A0008E008312603083168F0083120030831617
:1000B000910000008312C830831681008312313012
:1000C0009000003083168C00831210308B00612169
:1000D00081018E018F010B118B100B108C018B177E
:1000E0008420321986201221B40B8228031085192E
:1000F0000314BA0DF0303A02031968210F303A02A6
:10010000031964216C217028640008000800321172
:100110000130B7008B132030370783169B001C1467
:100120001A088312A4001030370783169B001C1492
:100130001A088312A3000030370783169B001C1493
:100140001A088312A2008B17331CAC28220903392A
:10015000A200A309A409A50901303702031DB5288F
:100160003E18B5283E143F14482101303702031DC4
:10017000BE283E1CBE283E103F144B21BF28B70AA4
:1001800002303702031808008A280130B600B40094
:10019000B500B70085018701B21357218420B40B45
:1001A000E228031085190314BA0DF0303A0203193E
:1001B0000029B51F8501B51F8701B50BE2289630D0
:1001C000B5000D21321DCE283211331CEC282D092B
:1001D0000339AD00AE09AF098B1320303707BC00DF
:1001E0002F08BB001B2110303707BC002E08BB00B6
:1001F0001B2100303707BC002D08BB001B218B17CB
:10020000850187015E21B70AB6010130B5000230D1
:100210003702031CCE286121080001303702031980
:100220004E2108003F1C08003F101030BC003E0863
:10023000BB001B2108008B133B0883161C159A007A
:1002400083123C0883169B0055309D00AA309D0008
:100250009C1464009C1829291C1183128B17080018
:10026000831610309B001C141A088312BE00FF3046
:10027000D4000230D5000C30D600BA30D700373069
:10028000D800DA30D9006F30DA00B830DB0008006F
:100290000130BE00080085018701080038093339A4
:1002A0008500B80039093F398700B90008001130CE
:1002B0008500B80013308700B9000800B801B90103
:1002C0000800BE013E1408003E143F1448210800F7
:1002D0003E103F144B21080001303E050319080071
:1002E0005C180516DC1885165C190514DC198514D4
:1002F0005C1A8714DC1A07155C1B0714DC1B8716B5
:100300005D180716DD188715E6300E02031C9229CA
:100310000516851605148514871407150714871606
:10032000071687158F08031908008F0185018701BB
:100330005408DE001F22D4005508DE001F22D5001D
:100340005608DE00541C1F22D6005708DE00D41CBD
:100350001F22D7005808DE00541D1F22D80059085C
:10036000DE00D41D1F22D9005A08DE00541E1F22B1
:10037000DA005B08DE00D41E1F22DB00CA0BC8298E
:100380005408CA00D4185C14D41E5C10D41D5C1030
:10039000CB0BD2295508CB00D51ADC14551DDC1027
:1003A000551FDC10CC0BDC295608CC00561A5C1506
:1003B000561F5C11D61D5C11CD0BE6295708CD00E8
:1003C000571ADC15D71FDC11D71DDC11CE0BF02915
:1003D0005808CE00D81B5C16D81F5C12D81C5C12C3
:1003E000CF0BFA295908CF00591ADC16591EDC1216
:1003F000D91FDC12D00B042A5A08D000DA195C1776
:10040000DA1D5C135A1E5C13D10B0E2A5B08D10057
:100410005B1ADC175B1EDC13DB1FDC13D20B162A06
:100420005608D200D51B5D14D71F5D10D30B1E2AB2
:100430005708D300D61BDD14D81FDD100800C001FB
:10044000DE080319DE035E184014DE1A401440086B
:10045000C0015E1C4014DE1E4014C005C00C5E0CC2
:02046000080092
:084000000F000300070001009E
:02400E00CC33B1
:104200000100FF00FF00FF00FF00FF00FF00FF00B4
:10421000FF00FF00FF00FF00FF00FF00FF00FF00A6
:104220000100FF00FF00FF00FF00FF00FF00FF0094
:10423000FF00FF00FF00FF00FF00FF00FF00FF0086
:104240000100FF00FF00FF00FF00FF00FF00FF0074
:10425000FF00FF00FF00FF00FF00FF00FF00050060
:10426000FF00FF00FF00FF00FF00FF00FF00FF0056
:10427000FF00FF00FF00FF00FF00FF00FF00FF0046
:10428000FF00FF00FF00FF00FF00FF00FF00FF0036
:10429000FF00FF00FF00FF00FF00FF00FF00FF0026
:1042A000FF00FF00FF00FF00FF00FF00FF00FF0016
:1042B000FF00FF00FF00FF00FF00FF00FF00FF0006
:1042C000FF00FF00FF00FF00FF00FF00FF00FF00F6
:1042D000FF00FF00FF00FF00FF00FF00FF00FF00E6
:1042E000FF00FF00FF00FF00FF00FF00FF00FF00D6
:1042F000FF00FF00FF00FF00FF00FF00FF000000C5
:00000001FF
